:100000000C945C000C9428040C9455040C9484000B
:100010000C9484000C9484000C9484000C94840050
:100020000C9484000C9484000C9484000C94840040
:100030000C9484000C9484000C9484000C94840030
:100040000C9482040C9484000C9484060C94840018
:100050000C9484000C9484000C9484000C94840010
:100060000C9484000C948400000024272A000025AE
:10007000282B000023262904040404040404040299
:100080000202020202030303030303010204081035
:100090002040800102040810200102040810200002
:1000A0000000070002010000030406000000000039
:1000B00000000000F4011A0311241FBECFEFD4E0AA
:1000C000DEBFCDBF11E0A0E0B1E0E8E9FEE002C094
:1000D00005900D92A433B107D9F711E0A4E3B1E084
:1000E00001C01D92A53FB107E1F710E0C8EBD0E0D9
:1000F00004C02297FE010E944607C43BD107C9F7FE
:100100000E9413030C944A070C940000FC01108217
:100110008FEF81831382128282E2848386E9858352
:10012000178216820895EF92FF920F931F93CF9339
:10013000DF93EC019B0177FF03C020E030E005C0B6
:10014000653B710514F024EB30E02983EC806D8170
:1001500070E06E197109882777FD8095982F982F88
:10016000872F762F662730E040E050E00E94C106DE
:1001700024EB30E040E050E00E941507FF2400E04F
:1001800010E0102F0F2DFE2CEE24E20EF31E041FA4
:10019000151FC801B70120E430E040E050E00E94A4
:1001A00015073B832A83DF91CF911F910F91FF9019
:1001B000EF9008955F926F927F928F929F92AF928D
:1001C000BF92CF92DF92EF92FF920F931F93DF9334
:1001D000CF93CDB7DEB76DB67EB6ADB65EB60E9434
:1001E000F20420913601309137014091380150914D
:1001F0003901621773078407950750F02C5E3F4F53
:100200004F4F5F4F621773078407950708F4AFC01D
:1002100060933601709337018093380190933901D0
:10022000E0913401F0913501BB2408C082819381B3
:10023000892B09F0B3940680F781E02D3097B1F750
:10024000BB2009F494C08B2D90E0880F991F2DB727
:100250003EB7281B390B0FB6F8943EBF0FBE2DBF1B
:10026000CDB6DEB60894C11CD11CA0913401B0916A
:10027000350120E013C012968D919C911397892B24
:1002800049F0E22FF0E0EE0FFF1FEC0DFD1DB183F2
:10029000A0832F5F16960D90BC91A02D109759F753
:1002A0002CC0812F90E07C01EE0CFF1CEC0CFD1C9F
:1002B000D7016D917C91FC013197EE0FFF1FEC0D82
:1002C000FD1D40815181DB0112962D913C911397C8
:1002D000DA0112968D919C9113972817390730F403
:1002E000D7014D935C937183608301E01F5F1B1501
:1002F000C0F2002311F410E011C011E000E0F7CFCC
:10030000E12FF0E0EE0FFF1FEC0DFD1D0190F081DD
:10031000E02D61E080810E94F8051F5F1B1580F3CE
:10032000F6B4EE2400E010E08F2C99241EC0EE2DD0
:10033000F0E0EE0FFF1FEC0DFD1D0190F081E02DB0
:1003400022813381280D391D86B58F1510F4005098
:100350001F4FF82EC8018F0D911D28173907A0F7E0
:1003600060E080810E94F805E394EB1400F38A2D8D
:10037000952D9C010FB6F8943EBF0FBE2DBF0FB652
:10038000F8947EBE0FBE6DBECF91DF911F910F918D
:10039000FF90EF90DF90CF90BF90AF909F908F90A5
:1003A0007F906F905F9008950F931F938C01FC01D5
:1003B00060838FEF81831382128280913401909148
:1003C000350197838683109335010093340160E0F3
:1003D00080810E94F80561E0F80180810E94DA05C1
:1003E00081E01F910F9108958AE391E00E948600B9
:1003F00082E491E00E9486008AE491E00E948600F7
:1004000008956BE570E08AE391E00E9493006AE54D
:1004100070E082E491E00E949300089581E010C0B2
:1004200070E08AE491E00E9493000E94DA006FE09D
:1004300070E080E090E00E94000580915C018F5F99
:1004400080935C0160915C01653B50F384EB10C0CC
:1004500070E08AE491E00E9493000E94DA006FE06D
:1004600070E080E090E00E94000580915C01815086
:1004700080935C0160915C01662351F7089540E828
:1004800055E260E070E08FE591E00E94250364E6AC
:1004900070E080E090E00E94000560E070E08091F4
:1004A0001D010E9482056091290170912A018AE351
:1004B00091E00E94D40160912B0170912C0182E4A3
:1004C00091E00E94D40160912101709122018AE49F
:1004D00091E00E94D4010E9401026DE570E08AE47F
:1004E00091E00E94930061E080911B010E94DA0577
:1004F00061E080911D010E94DA0561E080911F0199
:100500000E94DA0560E08EE00E94DA0560E08FE08C
:100510000E94DA0560E080E10E94DA0560E081E196
:100520000E94DA0561E08EE00E94F80561E08FE04C
:100530000E94F80561E080E10E94F80561E081E138
:100540000E94F805809152010E94640581509240FA
:100550003CF080E190E0909355018093540104C0F9
:100560001092550110925401809123010E9464055C
:10057000815092403CF080E290E09093570180934C
:10058000560104C010925701109256018091250126
:100590000E946405815092403CF080E490E090938A
:1005A00059018093580104C01092590110925801CA
:1005B000809127010E946405815092403CF080E8C0
:1005C00090E090935B0180935A0104C010925B010C
:1005D00010925A0180915601909157012091540137
:1005E00030915501820F931F20915801309159018C
:1005F000820F931F20915A0130915B01820F931F4C
:1006000090935E0180935D0160E071E08FE591E081
:100610000E942A0360915D0170915E018FE591E077
:100620000E94180408950E942A050E943F020E9419
:100630000E02FDCF82E391E09093600180935F0111
:100640000895862F0E947C060895CB01BA010E946E
:10065000430608950F931F93CF93DF938C01EB0113
:1006600009C02196D801ED91FC910190F081E02D17
:10067000C801099568816623A1F7DF91CF911F9189
:100680000F9108950F931F938C01DC01ED91FC9164
:100690000190F081E02D6DE00995D801ED91FC917C
:1006A0000190F081E02D6AE0C80109951F910F913A
:1006B00008952F923F924F925F926F927F928F9206
:1006C0009F92AF92BF92CF92DF92EF92FF920F93E1
:1006D0001F93DF93CF93CDB7DEB7A0970FB6F894F3
:1006E000DEBF0FBECDBF1C016A017B014115510564
:1006F0006105710549F4DC01ED91FC910190F081F7
:10070000E02D60E3099554C0882499245401422EB9
:1007100055246624772401E010E00C0F1D1F080DFE
:10072000191DC701B601A30192010E94F306F80149
:1007300060830894811C911CA11CB11CC701B601E7
:10074000A30192010E94F306C901DA016C017D0147
:10075000C114D104E104F104F1F681E0E82EF12C9A
:10076000EC0EFD1EE80CF91C3E010894611C711C86
:10077000D501C4010197A109B1096C01C818D908B4
:1007800014C0F601EE0DFF1D60816A3010F4605D4B
:1007900001C0695CD101ED91FC910190F081E02DE7
:1007A000C10109950894E108F1086E147F0449F726
:1007B000A0960FB6F894DEBF0FBECDBFCF91DF91EC
:1007C0001F910F91FF90EF90DF90CF90BF90AF906F
:1007D0009F908F907F906F905F904F903F902F9061
:1007E0000895EF92FF920F931F93CF93DF93EC0145
:1007F0007A018B0177FF0FC0E881F9810190F081C8
:10080000E02D6DE2099510950095F094E094E11CBF
:10081000F11C011D111D2AE0B801A701CE010E94A3
:100820005903DF91CF911F910F91FF90EF900895A1
:100830000F931F938C01AB01662757FD6095762FB0
:100840000E94F103C8010E9442031F910F91089575
:100850001F920F920FB60F9211242F933F934F9335
:100860005F936F937F938F939F93AF93BF93EF9318
:10087000FF938091610190916201892B29F0E091B1
:100880006101F09162010995FF91EF91BF91AF91E4
:100890009F918F917F916F915F914F913F912F9198
:1008A0000F900FBE0F901F9018951F920F920FB6CA
:1008B0000F9211242F933F934F935F936F937F93E6
:1008C0008F939F93AF93BF93EF93FF9380916301B7
:1008D00090916401892B29F0E0916301F09164010A
:1008E0000995FF91EF91BF91AF919F918F917F916A
:1008F0006F915F914F913F912F910F900FBE0F908D
:100900001F9018951F920F920FB60F9211242F93DC
:100910008F939F93AF93BF938091650190916601F0
:10092000A0916701B09168010196A11DB11D80934E
:10093000650190936601A0936701B093680180916F
:10094000690190916A01A0916B01B0916C01805096
:10095000904CAF4FBF4F8093690190936A01A09371
:100960006B01B0936C0127C08091690190916A017D
:10097000A0916B01B0916C0180589E43A040B040A3
:100980008093690190936A01A0936B01B0936C010D
:1009900080916D0190916E01A0916F01B0917001F5
:1009A0000196A11DB11D80936D0190936E01A093DE
:1009B0006F01B09370018091690190916A01A091DB
:1009C0006B01B0916C0181589E43A040B04060F62D
:1009D000BF91AF919F918F912F910F900FBE0F906C
:1009E0001F9018958FB7F89420916D0130916E018A
:1009F00040916F01509170018FBFB901CA010895F4
:100A0000EF92FF920F931F937B018C018FB7F894A5
:100A100040916D0150916E0160916F017091700174
:100A20008FBF2FB7F89480916D0190916E01A091C6
:100A30006F01B09170012FBF841B950BA60BB70BF4
:100A4000E816F9060A071B0760F71F910F91FF9040
:100A5000EF900895789484B5826084BD84B58160F8
:100A600084BD85B5826085BD85B5816085BDEEE6B6
:100A7000F0E0808181608083E1E8F0E08081826045
:100A80008083808181608083E0E8F0E08081816004
:100A90008083E1EBF0E0808184608083E0EBF0E034
:100AA000808181608083EAE7F0E0808184608083D8
:100AB0008081826080838081816080838081806882
:100AC00080831092C10008958F7090912D019295AE
:100AD000990F990F907C982B90937C0080917A00CD
:100AE000806480937A0080917A0086FDFCCF20910B
:100AF000780040917900942F80E030E0282B392B4A
:100B0000C90108951F93CF93DF93182FEB0161E084
:100B10000E94DA05E12FF0E0E156FF4F8491833027
:100B200051F480918000806880938000D093890088
:100B3000C09388003BC0843051F480918000806273
:100B400080938000D0938B00C0938A002FC08130A7
:100B500039F4209729F184B5806884BDC7BD26C0CB
:100B6000823039F42097E1F084B5806284BDC8BD3D
:100B70001DC0863041F48091B00080688093B00041
:100B8000C093B30013C0873041F48091B0008062FD
:100B90008093B000C093B40009C0C038D10514F4EC
:100BA00060E001C061E0812F0E94F805DF91CF91E4
:100BB0001F910895282F30E0C90185579F4FFC01F0
:100BC000949129583F4FF9018491882381F0E82FAF
:100BD000F0E0E859FF4FE491F0E0662329F48081CA
:100BE00090958923808308958081892B808308953F
:100BF000482F50E0CA0181569F4FFC012491CA0141
:100C000085579F4FFC01949149585F4FFA013491E9
:100C10003323C1F1222331F1233021F4809180006C
:100C20008F7705C0243031F4809180008F7D8093D0
:100C3000800018C0213019F484B58F7704C02230A9
:100C400021F484B58F7D84BD0DC0263021F48091C0
:100C5000B0008F7705C0273029F48091B0008F7DD8
:100C60008093B000E32FF0E0E359FF4FE491F0E010
:100C7000662329F48081909589238083089580815B
:100C8000892B80830895EF92FF920F931F937B012E
:100C90008C0122E030E040E050E00E941507205C2B
:100CA0003D4B404F5F4FCA01B901A80197010E9417
:100CB0001507C901DA010197A109B109292F3A2FB6
:100CC0004B2F552747FD5A950196A11DB11D209325
:100CD000C50081508093C400E1ECF0E08081806128
:100CE00080838081886080838081806880831F9179
:100CF0000F91FF90EF900895982F8091C00085FF8D
:100D0000FCCF9093C60008951F920F920FB60F92DA
:100D100011242F933F934F935F936F937F938F9300
:100D20009F93AF93BF93EF93FF934091C600E091E1
:100D30007101F0917201CF01019660E870E00E94AC
:100D4000E0069C0180917301909174012817390786
:100D500039F0EB58FE4F40833093720120937101BC
:100D6000FF91EF91BF91AF919F918F917F916F9183
:100D70005F914F913F912F910F900FBE0F901F9059
:100D80001895629FD001739FF001829FE00DF11DC5
:100D9000649FE00DF11D929FF00D839FF00D749FF5
:100DA000F00D659FF00D9927729FB00DE11DF91FA1
:100DB000639FB00DE11DF91FBD01CF0111240895FE
:100DC00097FB092E07260AD077FD04D049D006D01C
:100DD00000201AF4709561957F4F0895F6F790956D
:100DE00081959F4F0895A1E21A2EAA1BBB1BFD01FE
:100DF0000DC0AA1FBB1FEE1FFF1FA217B307E407FA
:100E0000F50720F0A21BB30BE40BF50B661F771F51
:100E1000881F991F1A9469F7609570958095909531
:100E20009B01AC01BD01CF01089597FB092E05265A
:100E30000ED057FD04D0D7DF0AD0001C38F45095EF
:100E40004095309521953F4F4F4F5F4F0895F6F7EE
:100E500090958095709561957F4F8F4F9F4F089526
:100E6000AA1BBB1B51E107C0AA1FBB1FA617B707D0
:100E700010F0A61BB70B881F991F5A95A9F78095EC
:100E80009095BC01CD010895EE0FFF1F0590F491E0
:080E9000E02D0994F894FFCF56
:100E9800486F6C612C20736F7920656C20726F62CB
:100EA8006F74206E756D65726F200006000B000868
:100EB80000030001000200030009000A000100000D
:040EC8000000210302
:00000001FF
